:020000020000FC
:020000003FC0FF
:02001000C5C168
:02002C0016C1FB
:02004800A3C053
:02004C00D5C01D
:10008000F1E0E0E0DD24D192F930E9F7E030D9F792
:1000900021E02093F80120E02093F9012FE0209344
:1000A000FA0128E02093FB0129E12093FC0123E1E0
:1000B0002093FD012FE02093FE0128E02EBF2FEFBB
:1000C0002DBF2FE224B92EE32AB920E42BB9D5B8ED
:1000D000D7B82FE328B900271127992488242FE3C4
:1000E0002093C7012093C80131D60E94170E0E94A9
:1000F0006E0B10D43FD0789430D63AD40ED010FF87
:10010000FBCF0E946D0E95D041D127D60E94920E52
:100110000E9489062DD401D0F8CF3091E405332315
:1001200021F021EA10D4D092E4053091E505332383
:1001300021F022EA08D4D092E5053091E605332378
:1001400021F023EA00D4D092E6053091E70533236D
:1001500021F024EAF8D3D092E70508955A9B02C013
:100160005A9808955A9A08955B9B02C05B98089527
:100170005B9A089527E62093C40028E9086020933D
:10018000C100CC240895D092C100089505601FC01D
:100190002F932FB72F93AF93BF93A091C0002091BF
:1001A000C600A97199F7203208F411C002FD16C0EB
:1001B000A0914603B0914703BA1779F0B8E02D93A8
:1001C000AF77A09346032B33A9F0243299F0BF9167
:1001D000AF912F912FBF2F91189506602B3311F0FF
:1001E0002432A9F7B8E0A0914603AA95AF7724E29C
:1001F0002C930B7FC394EBCF2F932FB72F93AF93F9
:10020000BF93B0914903A0914A03BA1769F0B3E0D4
:100210002D912093C600AF71A0934A03BF91AF9177
:100220002F912FBF2F911895086028E92093C100C6
:10023000F5CF2FE1209389002FE320938800D092FF
:10024000800029E02093810022E020936F00089530
:10025000D0928100D0926F0008952F932FB72F93E3
:1002600013FD08C0209144032D110DC02F912FBF05
:100270002F911895209145032A952093450391F7D6
:100280001460177FEFCF3F934F935F93FF93EF93EC
:1002900030914F034E2D20FF0FC0E0913803F091B5
:1002A00039033197E0933803F093390329F42E7F13
:1002B000106130FF41603E7F21FF0FC0E0913A03A3
:1002C000F0913B033197E0933A03F0933B0329F419
:1002D0002D7F106131FF42603D7F22FF0FC0E09112
:1002E0003C03F0913D033197E0933C03F0933D03D1
:1002F00029F42B7F106132FF44603B7F23FF0FC046
:10030000E0913E03F0913F033197E0933E03F09379
:100310003F0329F4277F106133FF4860377F24FFB4
:100320000FC0E0914003F09141033197E093400307
:10033000F093410329F42F7E106134FF40613F7E2A
:1003400025FF0FC0E0914203F09143033197E09302
:100350004203F093430329F42F7D106135FF40627F
:100360003F7D2093440330934F03E42EEF91FF91A0
:1003700014FD1AC05F914F913F912F912FBF2F9184
:100380001895D0926800D0926C000895F89422E0FD
:10039000209368002FE320936C00F8942F932FB7DD
:1003A0002F933F934F935F936F9366B130914E03BA
:1003B0003095262F2323509144033E2D352B309525
:1003C00040915F033423322330FF0AC0409153032E
:1003D00040933803409154034093390351602E7F7A
:1003E00031FF0AC04091550340933A0340915603B0
:1003F00040933B0352602D7F32FF0AC04091570368
:1004000040933C034091580340933D0354602B7F3D
:1004100033FF0AC04091590340933E0340915A0371
:1004200040933C035860277F34FF0AC040915B0330
:100430004093400340915C0340933D0350612F7E05
:1004400035FF0AC040915D034093420340915E0333
:100450004093430350622F7D30914D0340914F03F1
:10046000432B242B5F935E2D522B50FD04C0309103
:10047000B201432B232B51FD04C03091B301432B18
:10048000232B52FD04C03091B401432B232B53FD89
:1004900004C03091B501432B232B54FD04C030918F
:1004A000B601432B232B55FD04C03091B701432BDC
:1004B000232B20FD04C03091B201432B232B21FDBF
:1004C00004C03091B301432B232B22FD04C0309193
:1004D000B401432B232B23FD04C03091B501432BE2
:1004E000232B24FD04C03091B601432B232B25FD83
:1004F00004C03091B701432B232B30914E03432B83
:100500005091D0014093D0013F91642B362330931A
:1005100044033E2DE22E2095232309F4EEC13F93A0
:1005200020FF50C03091E40760918407362B609122
:10053000B40736233093E4073091E50760918507CF
:10054000362B6091B50736233093E5073091E607E7
:1005500060918607362B6091B60736233093E60705
:100560003091E70760918707362B6091B7073623F4
:100570003093E7073091E80760918807362B609148
:10058000B80736233093E8073091E907609189076F
:10059000362B6091B90736233093E9073091EA078B
:1005A00060918A07362B6091BA0736233093EA07A9
:1005B0003091EB0760918B07362B6091BB07362398
:1005C0003093EB0721FF50C03091E40760918C0716
:1005D000362B6091BC0736233093E4073091E50752
:1005E00060918D07362B6091BD0736233093E50768
:1005F0003091E60760918E07362B6091BE07362357
:100600003093E6073091E70760918F07362B6091B2
:10061000BF0736233093E7073091E80760919007D2
:10062000362B6091C00736233093E8073091E907F5
:1006300060919107362B6091C10736233093E9070B
:100640003091EA0760919207362B6091C2073623FA
:100650003093EA073091EB0760919307362B609156
:10066000C30736233093EB0722FF50C03091E407D5
:1006700060919407362B6091C40736233093E407CA
:100680003091E50760919507362B6091C5073623B9
:100690003093E5073091E60760919607362B60911D
:1006A000C60736233093E6073091E7076091970736
:1006B000362B6091C70736233093E7073091E80760
:1006C00060919807362B6091C80736233093E8076E
:1006D0003091E90760919907362B6091C90736235D
:1006E0003093E9073091EA0760919A07362B6091C1
:1006F000CA0736233093EA073091EB0760919B07D6
:10070000362B6091CB0736233093EB0723FF50C085
:100710003091E40760919C07362B6091CC0736231B
:100720003093E4073091E50760919D07362B609187
:10073000CD0736233093E5073091E60760919E0799
:10074000362B6091CE0736233093E6073091E707CA
:1007500060919F07362B6091CF0736233093E707D0
:100760003091E8076091A007362B6091D0073623BF
:100770003093E8073091E9076091A107362B60912B
:10078000D10736233093E9073091EA076091A20739
:10079000362B6091D20736233093EA073091EB076E
:1007A0006091A307362B6091D30736233093EB0774
:1007B00024FF50C03091E4076091A407362B60916C
:1007C000D40736233093E4073091E5076091A507FD
:1007D000362B6091D50736233093E5073091E60735
:1007E0006091A607362B6091D60736233093E60733
:1007F0003091E7076091A707362B6091D707362322
:100800003093E7073091E8076091A807362B609195
:10081000D80736233093E8073091E9076091A9079C
:10082000362B6091D90736233093E9073091EA07D8
:100830006091AA07362B6091DA0736233093EA07D6
:100840003091EB076091AB07362B6091DB073623C5
:100850003093EB0725FF50C03091E4076091AC075F
:10086000362B6091DC0736233093E4073091E5079F
:100870006091AD07362B6091DD0736233093E50795
:100880003091E6076091AE07362B6091DE07362384
:100890003093E6073091E7076091AF07362B609100
:1008A000DF0736233093E7073091E8076091B00700
:1008B000362B6091E00736233093E8073091E90743
:1008C0006091B107362B6091E10736233093E90739
:1008D0003091EA076091B207362B6091E207362328
:1008E0003093EA073091EB076091B307362B6091A4
:1008F000E30736233093EB073F916F91E3122BC749
:1009000014FF451328C75F914F913F912F912FBF3F
:100910002F91189520E02093490320934A0324E067
:1009200020934B0320934C032FE3E22E2093C60128
:100930000895F0914B03E0914C03FE1B08F4F0582E
:10094000F03650F00895F0914B03E0914C03FE1BFC
:1009500008F4F058FF3759F0E0914B03F5E020839D
:10096000F7E03193E43809F4E4E0E0934B030895B1
:10097000D0914903C0914A03DC1B08F4D05EDA3001
:1009800008F700FDB4C101FDBBC1F0914B03E0913C
:100990004C03FE17B9F2E0914C03F5E02081F7E03B
:1009A0003191E43809F4E4E0E0934C03C091490349
:1009B000D3E0E0E2E29F2770F4E0E1EEE10DFD1DFF
:1009C000099408951EC022C037C03BC097C099C08B
:1009D000A3C0A4C0B2C00DC115C11DC125C12DC188
:1009E00035C13DC145C14DC1A4C054C1089508954C
:1009F000089508950895089508950895089508950F
:100A000008952FE361D1232F5FD15DC12AE35CD12B
:100A100021E35AD120E358D120E356D1309150033D
:100A20003A3034F020E323953A503A30E4F74CD191
:100A300020E3230F49D147C12EE210FD27E244D124
:100A400042C122E241D122E43FD136E0FE2DE091C5
:100A50004D0329E4E0FD03C022E5F0FF24E534D195
:100A6000F695E6953A95A9F7FEE3E0919901249170
:100A70002BD1E0919B01249127D1E0919D012491FC
:100A800023D1E0919F0124911FD1E091A1012491F4
:100A90001BD1E091A301249117D1E09198012491F9
:100AA00013D1E0919A0124910FD1E0919C012491FE
:100AB0000BD1E0919E01249107D1E091A0012491F6
:100AC00003D1E091A2012491FFD0E091A4012491EF
:100AD000FBD0E091A5012491F7D0E091A6012491EB
:100AE000F3D0E091A7012491EFD0E091A8012491E7
:100AF000EBD0E091A9012491E7D0E5C0E22F2CE3EF
:100B000002C0E22F2EE3E0D021E32E0FDDD0FEE382
:100B1000E32F2491D9D0D7C028E201C029E2D4D054
:100B200021E3E6E030FDD0D036952395EA95D1F764
:100B3000CAC022E2C9D029E4F2CF2CE7C5D0FEE337
:100B40003091B101E32FE295EF702491BDD0E32FF6
:100B5000EF70EE0FEE0F3091B00124E0239FE129FA
:100B60002491B2D0E32FEF732491AED03091AF0136
:100B7000E32FE695E6952491A7D0E32FE295E07365
:100B80003091AE01232F22952F70E22B24919CD01F
:100B9000E32FEF70EE0FEE0F3091AD0124E0239FB5
:100BA000E129249191D0E32FEF7324918DD03091DE
:100BB000AC01E32FE695E695249186D0E32FE295EC
:100BC000E0733091AB01232F22952F70E22B2491FB
:100BD0007BD0E32FEF70EE0FEE0F3091AA0124E0EF
:100BE000239FE129249170D0E32FEF7324916CD0DF
:100BF0006AC0E22F21E268D021E32E0F65D023E402
:100C000063D05DC0E22F21E25FD021E32E0F5CD0E4
:100C100023E65AD054C0E22F21E256D021E32E0F12
:100C200053D026E451D04BC0E22F21E24DD021E336
:100C30002E0F4AD023E548D042C0E22F21E244D013
:100C400021E32E0F41D026E63FD039C0E22F21E22A
:100C50003BD021E32E0F38D023E736D030C0E22F2F
:100C600021E232D020E32E0F2FD028E52DD02BC04B
:100C7000E22F21E229D021E32E0F26D021E424D037
:100C80001EC0E22F21E220D021E32E0F1DD021E64D
:100C90001BD015C0E0E3E20F23E216D02E2F14D0B4
:100CA0002DE212D001D00FC0232F229502D0232F86
:100CB00000C02F70205D2A3338F0295F05C0FEE3A5
:100CC000E32F249101D02BE34C2F2993CF71F8947B
:100CD00003FD04C0C0934903789408957894077F76
:100CE0002093C600C42F48EB4093C10008950E7FA7
:100CF000C0914903D3E02FE3E7DF23E4E5DFE3CF4F
:100D00000D7FC0914903D3E02FE3DEDF26E4DCDF73
:100D1000DACF4E2D5091C6015427B9F04093C60149
:100D200005FF13C0DD2750FF0CC020E340FF28E281
:100D30002D0FB1E0A8E9AD0FAD0F40FFA3953C9199
:100D4000F8DDD3954695569571F7089520E02093E8
:100D500046032FE7209347030895CC2009F4089514
:100D6000CA94D8E0C0914703C395CF7728812B332D
:100D700091F0243209F0F8CFC0934703089528E09A
:100D800035E5E1DD2091480320934703089528E0ED
:100D900031E4D9DDF7CFC0934803C091470398D41D
:100DA00027FDEDCF2052F6E0E8EDE20FFD1D09949E
:100DB000E6CF5EC07CC289C2E2CF9AC2C6C2F1C28F
:100DC000F4C201C30FC3DBCFDACFD9CFD8CF40C332
:100DD000D6CFD5CFD4CFD3CFD2CFD1CFD0CFCFCF07
:100DE000CECFCDCF4EC3CBCFCACFC9CFC8CFC7CFC1
:100DF000C8C3C5CFC4CFC3CFC2CFC1CFC0CFBFCF71
:100E0000BECFBDCFBCCFBBCFBACFB9CFB8CFB7CF96
:100E1000B6CFB5CFB4CFB3CFB2CFB1CFB0CFAFCFC6
:100E2000AECFADCFACCF49C34FC36AC36EC3BCC353
:100E3000A6CFA5CFA4CFA3CFA2CFA1CFA0CF9FCF26
:100E40009ECF9DCF9CCF9BCF9ACF99CF98CF97CF56
:100E500096CF95CF94CF93CF92CF91CF90CF8FCF86
:100E60008ECF8DCF8CCF8BCF77C389CF78C387CFF1
:100E700028E0B1E0AEEBDD922A95E9F729D42053C2
:100E8000273098F5722F24D42B3379F1422F20D4B8
:100E9000F0E4E22F349137FD7ACF1AD42B33B1F13D
:100EA000F4E4E22FA491A7FD72CFF2502491A25452
:100EB000EC91E22BEC93F1CFF1E0E4EAE70F308321
:100EC000FAE3E72F24913091D801322B3093D801E7
:100ED0001062770F770F770FF2E0E0ECE70F28E072
:100EE0003D9131932A95E1F7089551CFF1E0E0E08B
:100EF00028E0F8943D9131932A95E1F7789410FF1A
:100F0000089522D420E807FD1EDD0895AEEB772377
:100F100069F37A95483579F0413471F24234F9F148
:100F2000443509F479C0423509F49BC04335D1F00A
:100F3000433431F12CCFFAE3E72F34912091D601DD
:100F4000232B10FD2093D601770F770F770FF5E055
:100F5000E4E810FDE4EBE70F28E03D9131932A959A
:100F6000E1F70895F7E0E4E8770F770F770FE70FE1
:100F700028E0F8943D9131932A95E1F7789408950B
:100F8000F7E0E4EB770F770F770FE70F28E0F8949F
:100F90003D91309531932A95D9F778940895F3E0EF
:100FA000ECE2E70FE70F31933083F2E0D2E0E72F76
:100FB000E295CE2FE05AC85928E04D9149934193CC
:100FC0002A95D9F7FCE3E0EA71D0F3E0E0E6E30F1D
:100FD0003081F3E0E0EAE70FE70F208031804484BE
:100FE000558431933083222D231220D1331619F0EA
:100FF000232D23101BD1431629F0421419F0242D60
:10100000431014D1531639F0521429F0531419F027
:10101000252D54100BD10FC1F3E0EDE2E70FE70FE0
:101020003083F2E0E72FE295E85928E04D914193B3
:101030002A95E1F7FCE3E0E839D0F3E0E0E6E30FDE
:101040003081F3E0E1EAE70FE70F2080348430835A
:10105000222D2312EBD0331619F0232D2310E6D0C6
:10106000EAC0F3E0ECE2E70FE70F3083F2E0E72FAE
:10107000E295E05A28E04D9141932A95E1F7FCE38F
:10108000E0E914D0F3E0E0E6E30F3081F3E0E0EADA
:10109000E70FE70F208034843083222D2312C6D03F
:1010A000331619F0232D2310C1D0D2C0E70FE70F5C
:1010B000159081286090CA01109461206092CA0145
:1010C000149091286090CB01109461206092CB0124
:1010D000FAE3E72F64914091D201462B57D09CD080
:1010E00039D019F46095462360954093D201409120
:1010F000D301462B73D068D02DD019F460954623C8
:1011000060954093D3014091D401462B67D084D0A1
:1011100021D019F46095462360954093D401409105
:10112000D501462B47D078D015D019F460954623C9
:1011300060954093D5014091C90160954623609523
:101140000EF4462B4093C9012091C801242B209313
:10115000C7010895231451F428E049905190451493
:1011600029F42A95D1F7989468940895E89420E496
:10117000229DE32DF6E6E00DF11DD491F051C491CE
:10118000F0516490DA5F288126210895D3E0C0E20F
:10119000C70FC70F2880C72FC295C050D2E008954F
:1011A000F3E0E0E2E70FE70F3080E72FE295E05051
:1011B000F2E00895D3E0C1E2C70FC70F2880C72F20
:1011C000C295C85FD2E00895F3E0E1E2E70FE70FD0
:1011D0003080E72FE295E85FF2E00895D3E0CCE2BB
:1011E000C70FC70F2880C72FC295C05AD2E00895F5
:1011F000F3E0ECE2E70FE70F3080E72FE295E05AEB
:10120000F2E00895D3E0CDE2C70FC70F2880C72FC3
:10121000C295C859D2E00895F3E0EDE2E70FE70F79
:101220003080E72FE295E859F2E00895222311F08B
:10123000231771F40895232F222351F4D3E0C8EB30
:10124000C70FC70FD992FAE3E72F24912883089597
:10125000D3E0C0EAF3E0E8EB4427552761E000243F
:101260007990721619F4762E782047297B847216AD
:1012700019F4762E782047297990721631F4D082AD
:10128000D182762E792057290E2E7B84721619F47E
:10129000762E79205729EE5F660F66FFE1CF552342
:1012A00049F2002039F2E02D41935083089510D285
:1012B000223419F0293421F06ACD20E23ADB62CDE4
:1012C00028E93091CE0135DB5DCD02D2283531F0F1
:1012D000D2D1B8F0308120EA36DB0895F894E8D412
:1012E0000E94C3000E9428014CD82CD20C94003FCD
:1012F000EFD1203339F0213369F02334A9F02336BC
:10130000D9F045CDE0E0F4E022E8D192D1922A95DF
:10131000E1F738CDE0E0F4E022E83FEF319331939C
:101320002A95E1F72FCD0895B5D1EEF350F3BC5FC8
:101330002C91232B2C93F8CFADD1AEF310F3BC5FDF
:101340002C91309523232C93F7CFC2D1203339F041
:10135000213369F02634A1F02636D1F018CDE0E033
:10136000F6E022E8D192D1922A95E1F70BCDE0E0A8
:10137000F6E022E83FEF319331932A95E1F702CD71
:1013800089D18EF288F0BA5F2C91232B2C93F8CF61
:1013900081D14EF248F0BA5F2C91309523232C93E3
:1013A000F7CF28E1C6DAEECCF2CC68D1E8F3209191
:1013B0004D03322B30934D0328E306FDC4DA10FDB4
:1013C0000C94CD0108955AD178F320914D033095B6
:1013D000322330934D0320E406FDB5DA10FD0C9462
:1013E000CD01089575D12B33E1F3223511F412604C
:1013F000F9CF223719F41D7F8DD4F4CF213411F4A5
:101400000061F0CF213611F40F7EECCF243511F4BA
:101410000062E8CF243711F40F7DE4CF293411F4B2
:101420000064E0CF293611F40F7BDCCF203319F4B0
:10143000F8940C940000213311F41360D3CF2835B5
:1014400011F40068CFCF283711F40F77CBCF9FCCA2
:1014500033273ED12B33D9F3A22F10D1C0F32091E3
:10146000C801A73529F0A93491F73095322301C07E
:10147000322B3093C8012091C901322B3093C70120
:10148000089526D12B33B9F020532A3000F7022ECD
:101490001FD12B3349F020532A30C8F63AE0309D53
:1014A000020E16D12B3399F620915003201541F3EB
:1014B00000925003E9D320E146CA96D040F2E0936F
:1014C000CC01F093CD01089503D121532630D0F5FE
:1014D0002F938AD02F91B0F1D3E0C3E5C20FC20F92
:1014E000E993F99340915F03FE2BFAE3E22F3491E5
:1014F00011F0432B02C03095432340935F030895BE
:1015000090D000F1009252030895E2D0203321F4EC
:10151000D092CE011BD036CC213329F42FE3209377
:10152000CE0114D02FCC2F93A9D02F9158F04091F9
:10153000CE01253441F0293429F4309534233093F9
:10154000CE0104C024CC342B3093CE01A7D310FF9E
:10155000089510610C94CD0128E4EBD913CCB8D0D8
:101560002153263078F72F9389D02F9158F3FAE33F
:10157000E22F4491432331F7D1E0C2EBC20F3993FC
:101580000895A6D021532630E8F62F9377D02F91D7
:10159000C8F2FAE3E22F4491542F432399F6D1E0A5
:1015A000C8EBC20F3883089593D0203319F0233548
:1015B00041F0EDCBE0E6F3E020E4D1922A95E9F7A3
:1015C000E1CB86D02B33F1F1F0E4E22F349137FDFB
:1015D000DECB7ED0F0E4E22F249127FDD8CBF3E0E0
:1015E000E0E6E30F2083EDCFFF27EE2771D02B330A
:1015F000A9F020532A3080F43AE0E39FE02D412DFA
:10160000F39FF02DE20FF41F112031F4F83220F493
:10161000F73261F7E03150F308940895EE0FFF1FA1
:101620000895002455D02B3361F020532A30A0F7C1
:101630003AE0039E020E112079F7202D243690F314
:10164000EBCF000C0895EE27FF2742D02B33D1F3C8
:1016500020532A3030F02750203118F0205220310A
:10166000D8F6EE0FFF1FEE0FFF1FEE0FFF1FEE0F5E
:10167000FF1FE20FEACFEE27FF27E8CF332728D05E
:101680002B3361F22153263038F6FAE3E22F24910E
:10169000322BF5CF1DD02B33C1F0F0E4E22F349183
:1016A00037FDBACF15D0F0E4E22FE491E7FDB4CFD7
:1016B00020E4329FF6E6E00DF11DB491F051A491C3
:1016C000F0513491E894889408956894889408952A
:1016D000C395CF772881C0934703089521E52CBD9A
:1016E00028E04091CE0140954F7747FD5D9A47FF36
:1016F0005D98DEBC26D05C9A24D023D05C983DB5A2
:1017000037FFFDCF440F2A9581F723E025B920E864
:101710002093D101F1E0E8E9D3E0C0E22FE33CE01F
:10172000219329933A95E1F7F1E0E4EA36E0219339
:101730003A95E9F72FEFF7E0E4EB30E321933A95A0
:10174000E9F70895DCBC08952F932FB72F933F93AB
:101750004F935F93F894D5B822273091B801E0FEFB
:10176000232B3091B901E1FE232B3091BA01E2FE27
:10177000232B3091BB01E3FE232B3091BC01E4FE0F
:10178000232B3091BD01E5FE232B309107014091C1
:101790000F0120FD40916F01E0FE40911701342BB5
:1017A00040911F0121FD40917701E1FE4091270109
:1017B000342B40912F0122FD40917F01E2FE4091A8
:1017C0003701342B40913F0123FD40918701E3FE17
:1017D00040914701342B40914F0124FD40918F01EE
:1017E000E4FE40915701342B40915F0125FD40916B
:1017F0009701E5FE40916701342B4091EB07342BB4
:101800003EBD3093B1015C985091D10150955093F9
:10181000D10157FD5D9A57FF5D98309106014091C7
:101820000E0120FD40916E01E0FE40911601342B27
:1018300040911E0121FD40917601E1FE409126017B
:10184000342B40912E0122FD40917E01E2FE409119
:101850003601342B40913E0123FD40918601E3FE89
:1018600040914601342B40914E0124FD40918E0160
:101870005C9AE4FE40915601342B40915E0125FDB7
:1018800040919601E5FE40916601342B4091EA07B4
:10189000342B4DB547FFFDCF3EBD3093B0015C9872
:1018A00056FD5D9A56FF5D983091050140910D01FE
:1018B00020FD40916D01E0FE40911501342B4091D7
:1018C0001D0121FD40917501E1FE40912501342B60
:1018D00040912D0122FD40917D01E2FE40913501B4
:1018E000342B40913D0123FD40918D01E3FE409159
:1018F0004501342B40914D0124FD40918D015C9AAE
:10190000E4FE40915501342B40915D0125FD40914D
:101910009501E5FE40916501342B4091E907342B98
:101920004DB547FFFDCF3EBD3093AF015091D00183
:101930003091CE0153275C9855FD5D9A55FF5D9817
:101940003091040140910C0120FD40916C01E0FEBA
:1019500040911401342B40911C0121FD40917401F0
:10196000E1FE40912401342B40912C0122FD409155
:101970007C01E2FE40913401342B40913C0123FD77
:1019800040918401E3FE40914401342B40914C018D
:1019900024FD40918C015C9AE4FE40915401342B6B
:1019A00040915C0125FD40919401E5FE4091640168
:1019B000342B4091E807342B4DB547FFFDCF3EBD9A
:1019C0003093AE015C9854FD5D9A54FF5D98309160
:1019D000030140910B0120FD40916B01E0FE40911D
:1019E0001301342B40911B0121FD40917301E1FE55
:1019F00040912301342B40912B0122FD40917B012A
:101A0000E2FE40913301342B40913B0123FD409194
:101A10008301E3FE40914301342B40914B015C9ADA
:101A200024FD40918B01E4FE40915301342B409101
:101A30005B0125FD40919301E5FE40916301342B4C
:101A40004091E707342B4DB547FFFDCF3EBD3093A6
:101A5000AD015C9853FD5D9A53FF5D983091020192
:101A600040910A0120FD40916A01E0FE409112017F
:101A7000342B40911A0121FD40917201E1FE409109
:101A80002201342B40912A0122FD40917A01E2FE8D
:101A900040913201342B40913A0123FD4091820163
:101AA000E3FE40914201342B40914A0124FD4091D4
:101AB0008A015C9AE4FE40915201342B40915A0114
:101AC00025FD40919201E5FE40916201342B409149
:101AD000E607342B4DB547FFFDCF3EBD3093AC013B
:101AE0005C9852FD5D9A52FF5D98309101014091E2
:101AF000090120FD40916901E0FE40911101342B64
:101B00004091190121FD40917101E1FE40912101B7
:101B1000342B4091290122FD40917901E2FE409150
:101B20003101342B4091390123FD40918101E3FEC5
:101B300040914101342B4091490124FD409189019C
:101B40005C9AE4FE40915101342B4091590125FDEE
:101B500040919101E5FE40916101342B4091E507F0
:101B6000342B4DB547FFFDCF3EBD3093AB015C98A4
:101B700051FD5D9A51FF5D9830910001409108013F
:101B800020FD40916801E0FE40911001342B40910E
:101B9000180121FD40917001E1FE40912001342B9C
:101BA0004091280122FD40917801E2FE40913001F0
:101BB000342B4091380123FD40918001E3FE409198
:101BC0004001342B4091480124FD409188015C9AEA
:101BD000E4FE40915001342B4091580125FD409185
:101BE0009001E5FE40916001342B4091E407342BD5
:101BF0004DB547FFFDCF3EBD3093AA015C9850FD27
:101C00005D9A50FF5D983091CE0153275093D001DB
:101C100098DD5C9A1F7E5F914DB547FFFDCF4F91D8
:101C20003F9123E025B92F912FBF2F91189521E0E7
:101C30004DD0353541F422E049D03A3A21F423E041
:101C400045D0323071F021E035E538D022E03AEA73
:101C500035D023E032E032D020E133272FD020E20C
:101C60002DD020E133D030935103343608F03327A0
:101C70003093500320E22AD03093CF01303408F063
:101C800033273093CE0108952091510330915003B2
:101C90002317C9F33093510320E110C02091CF01E5
:101CA0003091CE01231779F33093CF0120E206C0A3
:101CB00020E032E403D0F999FECF0895F999FECFE0
:101CC000D2BC21BD30BDFA9AF99A0895F999FECF98
:101CD000D2BC21BDF89A30B50895F894D092D601BF
:101CE000F1E0E0E1B5E0A4E826E038E04D91419371
:101CF0003A95E1F738962A95C1F72FE32093D20160
:101D00002093D3012093D4012093D50124E1209383
:101D1000CC011ACD212F13FF07C0137FD0924E03A1
:101D20000C94CD0111FD13FD08957091D601772318
:101D3000B9F131E046E0552721E8632F67236E2192
:101D400041F1F8942E2C262219F1B5E0A4EBA50F51
:101D5000D5E0C4E8C50F68E02D9029926A95E1F7B7
:101D6000A850D2E0C8E0C50FC50F4E2EF1E0E0E16B
:101D7000E50FE50F68E02D903990232821926A95B0
:101D8000D1F7789407FD0E94A30430957323309512
:101D90007894330F585F4A95239579F67093D6015E
:101DA00012FD25C0282D292915FF01F1F3E0E8EBEC
:101DB00021E03091C701A82CB92CFE2C2B2C22221B
:101DC00069F02180322C332249F0322C3F20231439
:101DD00029F02094B22020802094A220EE5F220FD0
:101DE000203461F72A2D2B2911F415FF089522279D
:101DF0005A2D50FFD6C0F3E0ECE2E20F408130E410
:101E0000439FF6E61F0E203001F130912003A0FC25
:101E100030912C03F001E30FB491F051A491F051F3
:101E20003491BC5F4C91342391F530912103B0FC87
:101E300030912D03F001E30FB491F051A491F051D2
:101E40003491BC5F4C91342311F5223009F130916B
:101E50002203A1FC30912E03F001E30FB491F05165
:101E6000A491F0513491BC5F4C91342381F43091B2
:101E70002303B1FC30912F03F001E30FB491F05133
:101E8000A491F0513491BC5F4C91342309F072C19C
:101E9000243001F130912403A2FC30913003F00191
:101EA000E30FB491F051A491F0513491BC5F4C9187
:101EB000342369F730912503B2FC30913103F001EE
:101EC000E30FB491F051A491F0513491BC5F4C9167
:101ED0003423E9F6263001F130912603A3FC30913A
:101EE0003203F001E30FB491F051A491F051349119
:101EF000BC5F4C91342359F630912703B3FC3091E9
:101F00003303F001E30FB491F051A491F0513491F7
:101F1000BC5F4C91342311F5283009F1309128032E
:101F2000A4FC30913403F001E30FB491F051A4917B
:101F3000F0513491BC5F4C91342381F430912903EA
:101F4000B4FC30913503F001E30FB491F051A4914A
:101F5000F0513491BC5F4C91342309F00BC12A300D
:101F600001F130912A03A5FC30913603F001E30F13
:101F7000B491F051A491F0513491BC5F4C91342351
:101F800069F730912B03B5FC30913703F001E30F73
:101F9000B491F051A491F0513491BC5F4C91342331
:101FA000E9F6EF1412FF21F42E5F569511F021CFC0
:101FB00008955B2D222750FFD6C0F3E0EDE2E20F3B
:101FC000408130E4439FF6E61F0E203001F130914E
:101FD0002003A0FC30912C03F001E30FB491F051E9
:101FE000A491F0513491BC5F4C91342391F5309120
:101FF0002103B0FC30912D03F001E30FB491F051B7
:10200000A491F0513491BC5F4C91342311F52230EE
:1020100009F130912203A1FC30912E03F001E30F6E
:10202000B491F051A491F0513491BC5F4C913423A0
:1020300081F430912303B1FC30912F03F001E30FC1
:10204000B491F051A491F0513491BC5F4C91342380
:1020500009F090C0243001F130912403A2FC3091AA
:102060003003F001E30FB491F051A491F051349199
:10207000BC5F4C91342369F730912503B2FC309159
:102080003103F001E30FB491F051A491F051349178
:10209000BC5F4C913423E9F6263001F130912603E0
:1020A000A3FC30913203F001E30FB491F051A491FD
:1020B000F0513491BC5F4C91342359F63091270391
:1020C000B3FC30913303F001E30FB491F051A491CC
:1020D000F0513491BC5F4C91342311F5283009F153
:1020E00030912803A4FC30913403F001E30FB49144
:1020F000F051A491F0513491BC5F4C913423D1F54F
:1021000030912903B4FC30913503F001E30FB49111
:10211000F051A491F0513491BC5F4C91342309F0FB
:1021200029C02A3001F130912A03A5FC30913603F1
:10213000F001E30FB491F051A491F0513491BC5FE0
:102140004C913423B9F430912B03B5FC3091370313
:10215000F001E30FB491F051A491F0513491BC5FC0
:102160004C91342339F4EF1412FFC9F42E5F5695C5
:1021700079F121CF12FDF2CEEF1489F4CC2079F45D
:1021800021E0B21AAD08A820B92079F4AA2069F498
:1021900015FD2CC06090D70177240C94DB1B0895AB
:1021A0001B7FD0924E030C94CD0121CE2E2D209575
:1021B0002B21E1F070934E0320915203222329F04A
:1021C0002093450318600C94CD0114600C94CD014C
:1021D00012FD0CC0BB2029F06091C701762F7B2136
:1021E00029F37E2D70957B2109F0C4CF222751E081
:1021F00066247090D701F1E0E4EAE20F408130E418
:10220000439FF6E61F0E203001F130912003A0FC21
:1022100030912C03F001E30FB491F051A491F051EF
:102220003491BC5F4C91342391F530912103B0FC83
:1022300030912D03F001E30FB491F051A491F051CE
:102240003491BC5F4C91342311F5213009F1309168
:102250002203A1FC30912E03F001E30FB491F05161
:10226000A491F0513491BC5F4C91342381F43091AE
:102270002303B1FC30912F03F001E30FB491F0512F
:10228000A491F0513491BC5F4C91342309F089C082
:10229000223001F130912403A2FC30913003F0018F
:1022A000E30FB491F051A491F0513491BC5F4C9183
:1022B000342369F730912503B2FC30913103F001EA
:1022C000E30FB491F051A491F0513491BC5F4C9163
:1022D0003423E9F6233009F130912603A3FC309131
:1022E0003203F001E30FB491F051A491F051349115
:1022F000BC5F4C91342359F630912703B3FC3091E5
:102300003303F001E30FB491F051A491F0513491F3
:10231000BC5F4C91342309F044C0243001F130916A
:102320002803A4FC30913403F001E30FB491F05181
:10233000A491F0513491BC5F4C91342391F53091CC
:102340002903B4FC30913503F001E30FB491F0514F
:10235000A491F0513491BC5F4C91342311F5253098
:1023600009F130912A03A5FC30913603F001E30F07
:10237000B491F051A491F0513491BC5F4C9134234D
:1023800081F430912B03B5FC30913703F001E30F5A
:10239000B491F051A491F0513491BC5F4C9134232D
:1023A00009F0652A550F2395263009F024CF7624AD
:1023B0005091D801752A2090D5013090D2014090DB
:1023C000D3015090D4017727F8942E2D20952B21FE
:1023D00021F012FD02C07894089570FE33C060FCB5
:1023E00021C02091C002209368012091C102209356
:1023F00069012091C20220936A012091C3022093B7
:102400006B012091C40220936C012091C50220939E
:102410006D012091C60220936E012091C702209386
:102420006F0110C0D0926801D0926901D0926A0108
:10243000D0926B01D0926C01D0926D01D0926E015E
:10244000D0926F0171FE33C061FC21C02091C8029F
:10245000209370012091C902209371012091CA023A
:10246000209372012091CB02209373012091CC0222
:10247000209374012091CD02209375012091CE020A
:10248000209376012091CF022093770110C0D09243
:102490007001D0927101D0927201D0927301D092EA
:1024A0007401D0927501D0927601D092770172FEBC
:1024B00033C062FC21C02091D0022093780120918A
:1024C000D102209379012091D20220937A012091A8
:1024D000D30220937B012091D40220937C01209190
:1024E000D50220937D012091D60220937E01209178
:1024F000D70220937F0110C0D0927801D092790149
:10250000D0927A01D0927B01D0927C01D0927D0151
:10251000D0927E01D0927F0173FE33C063FC21C054
:102520002091D802209380012091D902209381012B
:102530002091DA02209382012091DB022093830113
:102540002091DC02209384012091DD0220938501FB
:102550002091DE02209386012091DF0220938701E3
:1025600010C0D0928001D0928101D0928201D0928D
:102570008301D0928401D0928501D0928601D092BD
:10258000870174FE33C064FC21C02091E0022093D7
:1025900088012091E102209389012091E202209399
:1025A0008A012091E30220938B012091E402209381
:1025B0008C012091E50220938D012091E602209369
:1025C0008E012091E70220938F0110C0D0928801E4
:1025D000D0928901D0928A01D0928B01D0928C0145
:1025E000D0928D01D0928E01D0928F0175FE33C0B2
:1025F00065FC21C02091E802209390012091E9021E
:10260000209391012091EA02209392012091EB0204
:10261000209393012091EC02209394012091ED02EC
:10262000209395012091EE02209396012091EF02D4
:102630002093970110C0D0929001D0929101D09236
:102640009201D0929301D0929401D0929501D092B0
:102650009601D0929701B0FE45C112FD02C020FC48
:1026600009C071602091CC01209338032091CD01E5
:1026700020933903232DA0FC252D20FFACC02091F1
:102680002D03209321032093990120916802209328
:10269000080230918405232B2093100120916902B8
:1026A0002093090230918505232B2093110120915D
:1026B0006A0220930A0230918605232B209312018F
:1026C00020916B0220930B0230918705232B2093DE
:1026D000130120916C0220930C0230918805232B6A
:1026E0002093140120916D0220930D0230918905F1
:1026F000232B2093150120916E0220930E0230911E
:102700008A05232B2093160120916F0220930F023C
:1027100030918B05232B20931701A0FE37C0209109
:102720002C03209320032093980120916002209392
:10273000000220930801209161022093010220935E
:102740000901209162022093020220930A01209144
:1027500063022093030220930B01209164022093D3
:10276000040220930C01209165022093050220931E
:102770000D01209166022093060220930E01209104
:1027800067022093070220930F01D5C020912003F8
:1027900020939801209100022093080120910102CA
:1027A000209309012091020220930A012091030243
:1027B00020930B012091040220930C01209105022B
:1027C00020930D012091060220930E012091070213
:1027D00020930F01B0C020912D032093210320935B
:1027E0009901209398012091680220930802209378
:1027F000080130918405232B209310012091690258
:10280000209309022093090130918505232B209301
:10281000110120916A0220930A0220930A0130914B
:102820008605232B2093120120916B0220930B022B
:1028300020930B0130918705232B209313012091C6
:102840006C0220930C0220930C0130918805232BFD
:102850002093140120916D0220930D0220930D010D
:1028600030918905232B2093150120916E0220932E
:102870000E0220930E0130918A05232B209316011E
:1028800020916F0220930F0220930F0130918B054E
:10289000232B20931701A0FE4EC020912C032093E0
:1028A0002003209160022093000220916102209376
:1028B0000102209162022093020220916302209380
:1028C0000302209164022093040220916502209368
:1028D0000502209166022093060220916702209350
:1028E000070229C0A0FE27C040FC19CF2091210378
:1028F0002093980120910802209308012091090259
:102900002093090120910A0220930A0120910B02D1
:1029100020930B0120910C0220930C0120910D02B9
:1029200020930D0120910E0220930E0120910F02A1
:1029300020930F01B2CFB1FE45C112FD02C021FCB0
:1029400009C072602091CC0120933A032091CD01FF
:1029500020933B03232DA1FC252D21FFACC020910A
:102960002F032093230320939B012091780220932F
:10297000180230918C05232B20932001209179029D
:102980002093190230918D05232B20932101209152
:102990007A0220931A0230918E05232B2093220174
:1029A00020917B0220931B0230918F05232B2093D3
:1029B000230120917C0220931C0230919005232B4F
:1029C0002093240120917D0220931D0230919105D6
:1029D000232B2093250120917E0220931E0230910B
:1029E0009205232B2093260120917F0220931F0222
:1029F00030919305232B20932701A1FE37C020910E
:102A00002E032093220320939A0120917002209399
:102A1000100220931801209171022093110220933B
:102A20001901209172022093120220931A01209121
:102A300073022093130220931B01209174022093B0
:102A4000140220931C0120917502209315022093FB
:102A50001D01209176022093160220931E012091E1
:102A600077022093170220931F01D5C020912203E3
:102A700020939A01209110022093180120911102B5
:102A8000209319012091120220931A012091130220
:102A900020931B012091140220931C012091150208
:102AA00020931D012091160220931E0120911702F0
:102AB00020931F01B0C020912F0320932303209364
:102AC0009B0120939A012091780220931802209371
:102AD000180130918C05232B20932001209179023D
:102AE000209319022093190130918D05232B2093F7
:102AF000210120917A0220931A0220931A01309129
:102B00008E05232B2093220120917B0220931B0210
:102B100020931B0130918F05232B209323012091BB
:102B20007C0220931C0220931C0130919005232BE2
:102B30002093240120917D0220931D0220931D01EA
:102B400030919105232B2093250120917E02209323
:102B50001E0220931E0130919205232B2093260103
:102B600020917F0220931F0220931F013091930533
:102B7000232B20932701A1FE4EC020912E032093EA
:102B80002203209170022093100220917102209361
:102B9000110220917202209312022091730220935D
:102BA0001302209174022093140220917502209345
:102BB000150220917602209316022091770220932D
:102BC000170229C0A1FE27C041FC19CF2091230381
:102BD00020939A0120911802209318012091190244
:102BE0002093190120911A0220931A0120911B02AF
:102BF00020931B0120911C0220931C0120911D0297
:102C000020931D0120911E0220931E0120911F027E
:102C100020931F01B2CFB2FE45C112FD02C022FCBB
:102C200009C074602091CC0120933C032091CD0118
:102C300020933D03232DA2FC252D22FFACC0209123
:102C400031032093250320939D0120918802209336
:102C5000280230919405232B209330012091890282
:102C60002093290230919505232B20933101209147
:102C70008A0220932A0230919605232B2093320159
:102C800020918B0220932B0230919705232B2093C8
:102C9000330120918C0220932C0230919805232B34
:102CA0002093340120918D0220932D0230919905BB
:102CB000232B2093350120918E0220932E023091F8
:102CC0009A05232B2093360120918F0220932F0207
:102CD00030919B05232B20933701A2FE37C0209112
:102CE00030032093240320939C01209180022093A1
:102CF0002002209328012091810220932102209319
:102D00002901209182022093220220932A012091FE
:102D100083022093230220932B012091840220938D
:102D2000240220932C0120918502209325022093D8
:102D30002D01209186022093260220932E012091BE
:102D400087022093270220932F01D5C020912403CE
:102D500020939C01209120022093280120912102A0
:102D6000209329012091220220932A0120912302FD
:102D700020932B012091240220932C0120912502E5
:102D800020932D012091260220932E0120912702CD
:102D900020932F01B0C0209131032093250320936D
:102DA0009D0120939C01209188022093280220936A
:102DB000280130919405232B209330012091890222
:102DC000209329022093290130919505232B2093EC
:102DD000310120918A0220932A0220932A01309106
:102DE0009605232B2093320120918B0220932B02F6
:102DF00020932B0130919705232B209333012091B1
:102E00008C0220932C0220932C0130919805232BC7
:102E10002093340120918D0220932D0220932D01C7
:102E200030919905232B2093350120918E02209318
:102E30002E0220932E0130919A05232B20933601E8
:102E400020918F0220932F0220932F0130919B0518
:102E5000232B20933701A2FE4EC0209130032093F4
:102E6000240320918002209320022091810220934C
:102E7000210220918202209322022091830220933A
:102E80002302209184022093240220918502209322
:102E9000250220918602209326022091870220930A
:102EA000270229C0A2FE27C042FC19CF209125038A
:102EB00020939C012091280220932801209129022F
:102EC0002093290120912A0220932A0120912B028C
:102ED00020932B0120912C0220932C0120912D0274
:102EE00020932D0120912E0220932E0120912F025C
:102EF00020932F01B2CFB3FE45C112FD02C023FCC7
:102F000009C078602091CC0120933E032091CD012F
:102F100020933F03232DA3FC252D23FFACC020913C
:102F200033032093270320939F012091980220933D
:102F3000380230919C05232B209340012091990267
:102F40002093390230919D05232B2093410120913C
:102F50009A0220933A0230919E05232B209342013E
:102F600020919B0220933B0230919F05232B2093BD
:102F7000430120919C0220933C023091A005232B19
:102F80002093440120919D0220933D023091A105A0
:102F9000232B2093450120919E0220933E023091E5
:102FA000A205232B2093460120919F0220933F02EC
:102FB0003091A305232B20934701A3FE37C0209116
:102FC00032032093260320939E01209190022093A8
:102FD00030022093380120919102209331022093F6
:102FE0003901209192022093320220933A012091DC
:102FF00093022093330220933B012091940220936B
:10300000340220933C0120919502209335022093B5
:103010003D01209196022093360220933E0120919B
:1030200097022093370220933F01D5C020912603B9
:1030300020939E012091300220933801209131028B
:10304000209339012091320220933A0120913302DA
:1030500020933B012091340220933C0120913502C2
:1030600020933D012091360220933E0120913702AA
:1030700020933F01B0C02091330320932703209376
:103080009F0120939E012091980220933802209363
:10309000380130919C05232B209340012091990207
:1030A000209339022093390130919D05232B2093E1
:1030B000410120919A0220933A0220933A013091E3
:1030C0009E05232B2093420120919B0220933B02DB
:1030D00020933B0130919F05232B209343012091A6
:1030E0009C0220933C0220933C013091A005232BAD
:1030F0002093440120919D0220933D0220933D01A5
:103100003091A105232B2093450120919E0220930D
:103110003E0220933E013091A205232B20934601CD
:1031200020919F0220933F0220933F013091A305FD
:10313000232B20934701A3FE4EC0209132032093FE
:103140002603209190022093300220919102209337
:103150003102209192022093320220919302209317
:1031600033022091940220933402209195022093FF
:1031700035022091960220933602209197022093E7
:10318000370229C0A3FE27C043FC19CF2091270393
:1031900020939E012091380220933801209139021A
:1031A0002093390120913A0220933A0120913B0269
:1031B00020933B0120913C0220933C0120913D0251
:1031C00020933D0120913E0220933E0120913F0239
:1031D00020933F01B2CFB4FE45C112FD02C024FCD2
:1031E00009C070612091CC01209340032091CD0152
:1031F00020934103232DA4FC252D24FFACC0209156
:103200003503209329032093A1012091A802209344
:1032100048023091A405232B209350012091A9024C
:10322000209349023091A505232B20935101209131
:10323000AA0220934A023091A605232B2093520123
:103240002091AB0220934B023091A705232B2093B2
:1032500053012091AC0220934C023091A805232BFE
:10326000209354012091AD0220934D023091A90585
:10327000232B209355012091AE0220934E023091D2
:10328000AA05232B209356012091AF0220934F02D1
:103290003091AB05232B20935701A4FE37C020911A
:1032A0003403209328032093A0012091A0022093AF
:1032B0004002209348012091A102209341022093D3
:1032C00049012091A2022093420220934A012091B9
:1032D000A3022093430220934B012091A402209348
:1032E000440220934C012091A50220934502209393
:1032F0004D012091A6022093460220934E01209179
:10330000A7022093470220934F01D5C020912803A4
:103310002093A00120914002209348012091410276
:10332000209349012091420220934A0120914302B7
:1033300020934B012091440220934C01209145029F
:1033400020934D012091460220934E012091470287
:1033500020934F01B0C0209135032093290320937F
:10336000A1012093A0012091A8022093480220935C
:1033700048013091A405232B209350012091A902EC
:1033800020934902209349013091A505232B2093D6
:1033900051012091AA0220934A0220934A013091C0
:1033A000A605232B209352012091AB0220934B02C0
:1033B00020934B013091A705232B2093530120919B
:1033C000AC0220934C0220934C013091A805232B92
:1033D000209354012091AD0220934D0220934D0182
:1033E0003091A905232B209355012091AE02209303
:1033F0004E0220934E013091AA05232B20935601B3
:103400002091AF0220934F0220934F013091AB05E2
:10341000232B20935701A4FE4EC020913403209308
:1034200028032091A002209340022091A102209322
:1034300041022091A202209342022091A3022093F4
:1034400043022091A402209344022091A5022093DC
:1034500045022091A602209346022091A7022093C4
:10346000470229C0A4FE27C044FC19CF209129039C
:103470002093A00120914802209348012091490205
:103480002093490120914A0220934A0120914B0246
:1034900020934B0120914C0220934C0120914D022E
:1034A00020934D0120914E0220934E0120914F0216
:1034B00020934F01B2CFB5FE45C112FD02C025FCDD
:1034C00009C070622091CC01209342032091CD016C
:1034D00020934303232DA5FC252D25FFACC020916F
:1034E000370320932B032093A3012091B80220934C
:1034F00058023091AC05232B209360012091B90232
:10350000209359023091AD05232B20936101209126
:10351000BA0220935A023091AE05232B2093620108
:103520002091BB0220935B023091AF05232B2093A7
:1035300063012091BC0220935C023091B005232BE3
:10354000209364012091BD0220935D023091B1056A
:10355000232B209365012091BE0220935E023091BF
:10356000B205232B209366012091BF0220935F02B6
:103570003091B305232B20936701A5FE37C020911E
:10358000360320932A032093A2012091B0022093B6
:103590005002209358012091B102209351022093B0
:1035A00059012091B2022093520220935A01209196
:1035B000B3022093530220935B012091B402209325
:1035C000540220935C012091B50220935502209370
:1035D0005D012091B6022093560220935E01209156
:1035E000B7022093570220935F01D5C020912A0390
:1035F0002093A20120915002209358012091510262
:10360000209359012091520220935A012091530294
:1036100020935B012091540220935C01209155027C
:1036200020935D012091560220935E012091570264
:1036300020935F01B0C02091370320932B03209388
:10364000A3012093A2012091B80220935802209355
:1036500058013091AC05232B209360012091B902D1
:1036600020935902209359013091AD05232B2093CB
:1036700061012091BA0220935A0220935A0130919D
:10368000AE05232B209362012091BB0220935B02A5
:1036900020935B013091AF05232B20936301209190
:1036A000BC0220935C0220935C013091B005232B77
:1036B000209364012091BD0220935D0220935D015F
:1036C0003091B105232B209365012091BE022093F8
:1036D0005E0220935E013091B205232B2093660198
:1036E0002091BF0220935F0220935F013091B305C8
:1036F000232B20936701A5FE4EC020913603209313
:103700002A032091B002209350022091B10220930D
:1037100051022091B202209352022091B3022093D1
:1037200053022091B402209354022091B5022093B9
:1037300055022091B602209356022091B7022093A1
:10374000570229C0A5FE27C045FC19CF20912B03A5
:103750002093A201209158022093580120915902F0
:103760002093590120915A0220935A0120915B0223
:1037700020935B0120915C0220935C0120915D020B
:1037800020935D0120915E0220935E0120915F02F3
:1037900020935F01B2CF20914F03272B20934F033B
:1037A00020914403272B209344031061137FD09270
:1037B0004E030E94CD0156E061E07727B3E0ACE212
:1037C000D3E0C0EA0090CA011090CB01282D262337
:1037D000F9F02A2161F4202D2623D1F4062A04FFD2
:1037E00017C028E53C91270F0E94A30411C004FFD5
:1037F0000FC0342D2B2D26232D11352D28E73623F0
:103800003D1120E73C91270F0E94A30428812C87BB
:10381000A395C395292D262331F12B2199F4212D30
:10382000262309F52F2D262321F42091C7012623D5
:10383000D1F4162A04FF17C020E53C91270F0E94FF
:10384000A30411C004FF0FC0332D2A2D26232D11F0
:10385000352D28E636233D1120E63C91270F0E94A6
:10386000A30428812C87A3957395660F5A9509F0B8
:10387000ADCF0092CA011092CB016092D701D092D5
:10388000D80104FF16C056E061E07727D1E0C4EA12
:10389000372D362341F0362128E83D1120E93881C3
:1038A000270F0E94A304C3957395660F5A9509F0DC
:1038B000EFCFA094B094F3E0E8EB20812A2121938C
:1038C00020812B212193E43CC1F71F7D8A209B207E
:0238D000089559
:083A00000102040810204080BF
:103C000000010002000400080010002000400080B5
:103C1000010101020104010801100120014001809D
:103C20000201020202040208021002200240028085
:103C3000030103020304030803100320034003806D
:103C40000401040204040408041004200440048055
:103C5000050105020504050805100520054005803D
:103C60000601060206040608061006200640068025
:103C7000070107020704070807100720074007800D
:103C800000010002000400080010002000000000F5
:103C900001000200040008001000200000000000E5
:103CA0000101020204040808101020200000000096
:103E00003031323334353637383941424344454610
:103E10004748494A4B4C4D4E4F50515253545556BA
:103E20005758595A6162636465666768696A6B6C62
:103E30006D6E6F707172737475767778797A7B7D39
:10400000FFFFFFFFFFFFFFFFFFFFFFFFFFFFFFFFC0
:10401000FFFFFFFFFFFFFFFFFFFFFFFFFFFFFFFFB0
:10402000FFFFFFFFFFFFFFFFFFFFFFFFFFFFFFFFA0
:1040300000010203040506070809FFFFFFFFFFFF59
:10404000FF0A0B0C0D0E0F10111213141516171872
:10405000191A1B1C1D1E1F20212223FFFFFFFFFF1B
:10406000FF2425262728292A2B2C2D2E2F303132CC
:10407000333435363738393A3B3C3D3EFF3FFFFF5E
:10408000FFFFFFFFFFFFFFFFFFFFFFFFFFFFFFFF40
:10409000FFFFFFFFFFFFFFFFFFFFFFFFFFFFFFFF30
:1040A000FFFFFFFFFFFFFFFFFFFFFFFFFFFFFFFF20
:1040B000FFFFFFFFFFFFFFFFFFFFFFFFFFFFFFFF10
:1040C000FFFFFFFFFFFFFFFFFFFFFFFFFFFFFFFF00
:1040D000FFFFFFFFFFFFFFFFFFFFFFFFFFFFFFFFF0
:1040E000FFFFFFFFFFFFFFFFFFFFFFFFFFFFFFFFE0
:1040F000FFFFFFFFFFFFFFFFFFFFFFFFFFFFFFFFD0
:10420000FFFFFFFFFFFFFFFFFFFFFFFFFFFFFFFFBE
:10421000FFFFFFFFFFFFFFFFFFFFFFFFFFFFFFFFAE
:10422000FFFFFFFFFFFFFFFFFFFFFFFFFFFFFFFF9E
:1042300001020408102040800102FFFFFFFFFFFF82
:10424000FF04081020408001020408102040800173
:104250000204081020408001020408FFFFFFFFFF56
:10426000FF10204080010204081020408001020459
:10427000081020408001020408102040FF80FFFF4A
:10428000FFFFFFFFFFFFFFFFFFFFFFFFFFFFFFFF3E
:10429000FFFFFFFFFFFFFFFFFFFFFFFFFFFFFFFF2E
:1042A000FFFFFFFFFFFFFFFFFFFFFFFFFFFFFFFF1E
:1042B000FFFFFFFFFFFFFFFFFFFFFFFFFFFFFFFF0E
:1042C000FFFFFFFFFFFFFFFFFFFFFFFFFFFFFFFFFE
:1042D000FFFFFFFFFFFFFFFFFFFFFFFFFFFFFFFFEE
:1042E000FFFFFFFFFFFFFFFFFFFFFFFFFFFFFFFFDE
:1042F000FFFFFFFFFFFFFFFFFFFFFFFFFFFFFFFFCE
:10440000FFFFFFFFFFFFFFFFFFFFFFFFFFFFFFFFBC
:10441000FFFFFFFFFFFFFFFFFFFFFFFFFFFFFFFFAC
:10442000FFFFFFFFFFFFFFFFFFFFFFFFFFFFFFFF9C
:1044300000000000000000000101FFFFFFFFFFFF80
:10444000FF01010101010102020202020202020354
:104450000303030303030304040404FFFFFFFFFF3C
:10446000FF04040404050505050505050506060603
:10447000060606060607070707070707FF07FFFFE9
:10448000FFFFFFFFFFFFFFFFFFFFFFFFFFFFFFFF3C
:10449000FFFFFFFFFFFFFFFFFFFFFFFFFFFFFFFF2C
:1044A000FFFFFFFFFFFFFFFFFFFFFFFFFFFFFFFF1C
:1044B000FFFFFFFFFFFFFFFFFFFFFFFFFFFFFFFF0C
:1044C000FFFFFFFFFFFFFFFFFFFFFFFFFFFFFFFFFC
:1044D000FFFFFFFFFFFFFFFFFFFFFFFFFFFFFFFFEC
:1044E000FFFFFFFFFFFFFFFFFFFFFFFFFFFFFFFFDC
:1044F000FFFFFFFFFFFFFFFFFFFFFFFFFFFFFFFFCC
:10460000010101010101010101010101010101019A
:10461000010101010101010101010101010101018A
:10462000010101010101010101010101010101017A
:10463000010101010101010101010101010101016A
:10464000010202020202020202020202020202024B
:10465000020202020202020202020202020202023A
:10466000020202020202020202020202020202022A
:10467000020202020202020202020202020202021A
:1046800001020404040404040404040404040404EF
:1046900004040404040404040404040404040404DA
:1046A00004040404040404040404040404040404CA
:1046B00004040404040404040404040404040404BA
:1046C000010204080808080808080808080808087B
:1046D000080808080808080808080808080808085A
:1046E000080808080808080808080808080808084A
:1046F000080808080808080808080808080808083A
:1047000001020408101010101010101010101010DA
:104710001010101010101010101010101010101099
:104720001010101010101010101010101010101089
:104730001010101010101010101010101010101079
:1047400001020408102020202020202020202020EA
:104750002020202020202020202020202020202059
:104760002020202020202020202020202020202049
:104770002020202020202020202020202020202039
:10478000010204081020404040404040404040406A
:104790004040404040404040404040404040404019
:1047A0004040404040404040404040404040404009
:1047B00040404040404040404040404040404040F9
:1047C00001020408102040808080808080808080EA
:1047D00080808080808080808080808080808080D9
:1047E00080808080808080808080808080808080C9
:1047F00080808080808080808080808080808080B9
:1048000001020408102040800101010101010101A1
:104810000101010101010101010101010101010188
:104820000101010101010101010101010101010178
:104830000101010101010101010101010101010168
:10484000010204081020408001020202020202025A
:104850000202020202020202020202020202020238
:104860000202020202020202020202020202020228
:104870000202020202020202020202020202020218
:10488000010204081020408001020404040404040E
:1048900004040404040404040404040404040404D8
:1048A00004040404040404040404040404040404C8
:1048B00004040404040404040404040404040404B8
:1048C00001020408102040800102040808080808BA
:1048D0000808080808080808080808080808080858
:1048E0000808080808080808080808080808080848
:1048F0000808080808080808080808080808080838
:104900000102040810204080010204081010101059
:104910001010101010101010101010101010101097
:104920001010101010101010101010101010101087
:104930001010101010101010101010101010101077
:1049400001020408102040800102040810202020E9
:104950002020202020202020202020202020202057
:104960002020202020202020202020202020202047
:104970002020202020202020202020202020202037
:104980000102040810204080010204081020404069
:104990004040404040404040404040404040404017
:1049A0004040404040404040404040404040404007
:1049B00040404040404040404040404040404040F7
:1049C00001020408102040800102040810204080E9
:1049D00080808080808080808080808080808080D7
:1049E00080808080808080808080808080808080C7
:1049F00080808080808080808080808080808080B7
:104A000001020408102040800102040810204080A8
:104A10000101010101010101010101010101010186
:104A20000101010101010101010101010101010176
:104A30000101010101010101010101010101010166
:104A40000102040810204080010204081020408068
:104A50000102020202020202020202020202020237
:104A60000202020202020202020202020202020226
:104A70000202020202020202020202020202020216
:104A80000102040810204080010204081020408028
:104A900001020404040404040404040404040404DB
:104AA00004040404040404040404040404040404C6
:104AB00004040404040404040404040404040404B6
:104AC00001020408102040800102040810204080E8
:104AD0000102040808080808080808080808080867
:104AE0000808080808080808080808080808080846
:104AF0000808080808080808080808080808080836
:104B000001020408102040800102040810204080A7
:104B100001020408101010101010101010101010C6
:104B20001010101010101010101010101010101085
:104B30001010101010101010101010101010101075
:104B40000102040810204080010204081020408067
:104B500001020408102020202020202020202020D6
:104B60002020202020202020202020202020202045
:104B70002020202020202020202020202020202035
:104B80000102040810204080010204081020408027
:104B90000102040810204040404040404040404056
:104BA0004040404040404040404040404040404005
:104BB00040404040404040404040404040404040F5
:104BC00001020408102040800102040810204080E7
:104BD00001020408102040808080808080808080D6
:104BE00080808080808080808080808080808080C5
:104BF00080808080808080808080808080808080B5
:104C000001020408102040800102040810204080A6
:104C1000010204081020408001010101010101018D
:104C20000101010101010101010101010101010174
:104C30000101010101010101010101010101010164
:104C40000102040810204080010204081020408066
:104C50000102040810204080010202020202020246
:104C60000202020202020202020202020202020224
:104C70000202020202020202020202020202020214
:104C80000102040810204080010204081020408026
:104C900001020408102040800102040404040404FA
:104CA00004040404040404040404040404040404C4
:104CB00004040404040404040404040404040404B4
:104CC00001020408102040800102040810204080E6
:104CD00001020408102040800102040808080808A6
:104CE0000808080808080808080808080808080844
:104CF0000808080808080808080808080808080834
:104D000001020408102040800102040810204080A5
:104D10000102040810204080010204081010101045
:104D20001010101010101010101010101010101083
:104D30001010101010101010101010101010101073
:104D40000102040810204080010204081020408065
:104D500001020408102040800102040810202020D5
:104D60002020202020202020202020202020202043
:104D70002020202020202020202020202020202033
:104D80000102040810204080010204081020408025
:104D90000102040810204080010204081020404055
:104DA0004040404040404040404040404040404003
:104DB00040404040404040404040404040404040F3
:104DC00001020408102040800102040810204080E5
:104DD00001020408102040800102040810204080D5
:104DE00080808080808080808080808080808080C3
:104DF00080808080808080808080808080808080B3
:104E000001020408102040800102040810204080A4
:104E10000102040810204080010204081020408094
:104E20008080808080808080808080808080808082
:104E30008080808080808080808080808080808072
:104E40000102040810204080010204081020408064
:104E50000102040810204080010204081020408054
:104E60008040404040404040404040404040404002
:104E70004040404040404040404040404040404032
:104E80000102040810204080010204081020408024
:104E90000102040810204080010204081020408014
:104EA0008040202020202020202020202020202082
:104EB00020202020202020202020202020202020F2
:104EC00001020408102040800102040810204080E4
:104ED00001020408102040800102040810204080D4
:104EE0008040201010101010101010101010101012
:104EF00010101010101010101010101010101010B2
:104F000001020408102040800102040810204080A3
:104F10000102040810204080010204081020408093
:104F20008040201008080808080808080808080831
:104F300008080808080808080808080808080808F1
:104F40000102040810204080010204081020408063
:104F50000102040810204080010204081020408053
:104F6000804020100804040404040404040404041D
:104F700004040404040404040404040404040404F1
:104F80000102040810204080010204081020408023
:104F90000102040810204080010204081020408013
:104FA00080402010080402020202020202020202F1
:104FB00002020202020202020202020202020202D1
:104FC00001020408102040800102040810204080E3
:104FD00001020408102040800102040810204080D3
:104FE00080402010080402010101010101010101BA
:104FF00001010101010101010101010101010101A1
:1050000001020408102040800102040810204080A2
:105010000102040810204080010204081020408092
:105020008040201008040201808080808080808081
:105030008080808080808080808080808080808070
:105040000102040810204080010204081020408062
:105050000102040810204080010204081020408052
:105060008040201008040201804040404040404001
:105070004040404040404040404040404040404030
:105080000102040810204080010204081020408022
:105090000102040810204080010204081020408012
:1050A0008040201008040201804020202020202081
:1050B00020202020202020202020202020202020F0
:1050C00001020408102040800102040810204080E2
:1050D00001020408102040800102040810204080D2
:1050E0008040201008040201804020101010101091
:1050F00010101010101010101010101010101010B0
:1051000001020408102040800102040810204080A1
:105110000102040810204080010204081020408091
:105120008040201008040201804020100808080870
:1051300008080808080808080808080808080808EF
:105140000102040810204080010204081020408061
:105150000102040810204080010204081020408051
:10516000804020100804020180402010080404043C
:1051700004040404040404040404040404040404EF
:105180000102040810204080010204081020408021
:105190000102040810204080010204081020408011
:1051A0008040201008040201804020100804020200
:1051B00002020202020202020202020202020202CF
:1051C00001020408102040800102040810204080E1
:1051D00001020408102040800102040810204080D1
:1051E00080402010080402018040201008040201C1
:1051F000010101010101010101010101010101019F
:1052000001020408102040800102040810204080A0
:105210000102040810204080010204081020408090
:105220008040201008040201804020100804020180
:10523000808080808080808080808080808080806E
:105240000102040810204080010204081020408060
:105250000102040810204080010204081020408050
:105260008040201008040201804020100804020140
:1052700080404040404040404040404040404040EE
:105280000102040810204080010204081020408020
:105290000102040810204080010204081020408010
:1052A0008040201008040201804020100804020100
:1052B000804020202020202020202020202020206E
:1052C00001020408102040800102040810204080E0
:1052D00001020408102040800102040810204080D0
:1052E00080402010080402018040201008040201C0
:1052F00080402010101010101010101010101010FE
:10530000010204081020408001020408102040809F
:10531000010204081020408001020408102040808F
:10532000804020100804020180402010080402017F
:10533000804020100808080808080808080808081D
:10534000010204081020408001020408102040805F
:10535000010204081020408001020408102040804F
:10536000804020100804020180402010080402013F
:105370008040201008040404040404040404040409
:10538000010204081020408001020408102040801F
:10539000010204081020408001020408102040800F
:1053A00080402010080402018040201008040201FF
:1053B00080402010080402020202020202020202DD
:1053C00001020408102040800102040810204080DF
:1053D00001020408102040800102040810204080CF
:1053E00080402010080402018040201008040201BF
:1053F00080402010080402010101010101010101A6
:10540000010204081020408001020408102040809E
:10541000010204081020408001020408102040808E
:10542000804020100804020180402010080402017E
:10543000804020100804020180808080808080806D
:10544000010204081020408001020408102040805E
:10545000010204081020408001020408102040804E
:10546000804020100804020180402010080402013E
:1054700080402010080402018040404040404040ED
:10548000010204081020408001020408102040801E
:10549000010204081020408001020408102040800E
:1054A00080402010080402018040201008040201FE
:1054B000804020100804020180402020202020206D
:1054C00001020408102040800102040810204080DE
:1054D00001020408102040800102040810204080CE
:1054E00080402010080402018040201008040201BE
:1054F000804020100804020180402010101010107D
:10550000010204081020408001020408102040809D
:10551000010204081020408001020408102040808D
:10552000804020100804020180402010080402017D
:10553000804020100804020180402010080808085C
:10554000010204081020408001020408102040805D
:10555000010204081020408001020408102040804D
:10556000804020100804020180402010080402013D
:105570008040201008040201804020100804040428
:10558000010204081020408001020408102040801D
:10559000010204081020408001020408102040800D
:1055A00080402010080402018040201008040201FD
:1055B00080402010080402018040201008040202EC
:1055C00001020408102040800102040810204080DD
:1055D00001020408102040800102040810204080CD
:1055E00080402010080402018040201008040201BD
:1055F00080402010080402018040201008040201AD
:1056000004080C1014181C2024282C3034383C407A
:1056100044484C5054585C6064686C7074787C806A
:1056200084888C9094989CA0A4A8ACB0B4B8BCC05A
:10563000C4C8CCD0D4D8DCE0E4E8ECF0F4F8FC004A
:1056400008080C1014181C2024282C3034383C4036
:1056500044484C5054585C6064686C7074787C802A
:1056600084888C9094989CA0A4A8ACB0B4B8BCC01A
:10567000C4C8CCD0D4D8DCE0E4E8ECF0F4F8FC000A
:105680000C0C0C1014181C2024282C3034383C40EE
:1056900044484C5054585C6064686C7074787C80EA
:1056A00084888C9094989CA0A4A8ACB0B4B8BCC0DA
:1056B000C4C8CCD0D4D8DCE0E4E8ECF0F4F8FC00CA
:1056C0001010101014181C2024282C3034383C40A2
:1056D00044484C5054585C6064686C7074787C80AA
:1056E00084888C9094989CA0A4A8ACB0B4B8BCC09A
:1056F000C4C8CCD0D4D8DCE0E4E8ECF0F4F8FC008A
:105700001414141414181C2024282C3034383C4051
:1057100044484C5054585C6064686C7074787C8069
:1057200084888C9094989CA0A4A8ACB0B4B8BCC059
:10573000C4C8CCD0D4D8DCE0E4E8ECF0F4F8FC0049
:105740001818181818181C2024282C3034383C40FD
:1057500044484C5054585C6064686C7074787C8029
:1057600084888C9094989CA0A4A8ACB0B4B8BCC019
:10577000C4C8CCD0D4D8DCE0E4E8ECF0F4F8FC0009
:105780001C1C1C1C1C1C1C2024282C3034383C40A5
:1057900044484C5054585C6064686C7074787C80E9
:1057A00084888C9094989CA0A4A8ACB0B4B8BCC0D9
:1057B000C4C8CCD0D4D8DCE0E4E8ECF0F4F8FC00C9
:1057C000202020202020202024282C3034383C4049
:1057D00044484C5054585C6064686C7074787C80A9
:1057E00084888C9094989CA0A4A8ACB0B4B8BCC099
:1057F000C4C8CCD0D4D8DCE0E4E8ECF0F4F8FC0089
:10580000242424242424242425292D3135393D41E0
:1058100045494D5155595D6165696D7175797D8158
:1058200085898D9195999DA1A5A9ADB1B5B9BDC148
:10583000C5C9CDD1D5D9DDE1E5E9EDF1F5F9FD0138
:10584000282828282828282829292D3135393D417C
:1058500045494D5155595D6165696D7175797D8118
:1058600085898D9195999DA1A5A9ADB1B5B9BDC108
:10587000C5C9CDD1D5D9DDE1E5E9EDF1F5F9FD01F8
:105880002C2C2C2C2C2C2C2C2D2D2D3135393D4114
:1058900045494D5155595D6165696D7175797D81D8
:1058A00085898D9195999DA1A5A9ADB1B5B9BDC1C8
:1058B000C5C9CDD1D5D9DDE1E5E9EDF1F5F9FD01B8
:1058C00030303030303030303131313135393D41A8
:1058D00045494D5155595D6165696D7175797D8198
:1058E00085898D9195999DA1A5A9ADB1B5B9BDC188
:1058F000C5C9CDD1D5D9DDE1E5E9EDF1F5F9FD0178
:1059000034343434343434343535353535393D4137
:1059100045494D5155595D6165696D7175797D8157
:1059200085898D9195999DA1A5A9ADB1B5B9BDC147
:10593000C5C9CDD1D5D9DDE1E5E9EDF1F5F9FD0137
:1059400038383838383838383939393939393D41C3
:1059500045494D5155595D6165696D7175797D8117
:1059600085898D9195999DA1A5A9ADB1B5B9BDC107
:10597000C5C9CDD1D5D9DDE1E5E9EDF1F5F9FD01F7
:105980003C3C3C3C3C3C3C3C3D3D3D3D3D3D3D414B
:1059900045494D5155595D6165696D7175797D81D7
:1059A00085898D9195999DA1A5A9ADB1B5B9BDC1C7
:1059B000C5C9CDD1D5D9DDE1E5E9EDF1F5F9FD01B7
:1059C00040404040404040404141414141414141CF
:1059D00045494D5155595D6165696D7175797D8197
:1059E00085898D9195999DA1A5A9ADB1B5B9BDC187
:1059F000C5C9CDD1D5D9DDE1E5E9EDF1F5F9FD0177
:105A0000444444444444444445454545454545454E
:105A1000464A4E52565A5E62666A6E72767A7E8246
:105A2000868A8E92969A9EA2A6AAAEB2B6BABEC236
:105A3000C6CACED2D6DADEE2E6EAEEF2F6FAFE0226
:105A400048484848484848484949494949494949CE
:105A50004A4A4E52565A5E62666A6E72767A7E8202
:105A6000868A8E92969A9EA2A6AAAEB2B6BABEC2F6
:105A7000C6CACED2D6DADEE2E6EAEEF2F6FAFE02E6
:105A80004C4C4C4C4C4C4C4C4D4D4D4D4D4D4D4D4E
:105A90004E4E4E52565A5E62666A6E72767A7E82BA
:105AA000868A8E92969A9EA2A6AAAEB2B6BABEC2B6
:105AB000C6CACED2D6DADEE2E6EAEEF2F6FAFE02A6
:105AC00050505050505050505151515151515151CE
:105AD00052525252565A5E62666A6E72767A7E826E
:105AE000868A8E92969A9EA2A6AAAEB2B6BABEC276
:105AF000C6CACED2D6DADEE2E6EAEEF2F6FAFE0266
:105B0000545454545454545455555555555555554D
:105B100056565656565A5E62666A6E72767A7E821D
:105B2000868A8E92969A9EA2A6AAAEB2B6BABEC235
:105B3000C6CACED2D6DADEE2E6EAEEF2F6FAFE0225
:105B400058585858585858585959595959595959CD
:105B50005A5A5A5A5A5A5E62666A6E72767A7E82C9
:105B6000868A8E92969A9EA2A6AAAEB2B6BABEC2F5
:105B7000C6CACED2D6DADEE2E6EAEEF2F6FAFE02E5
:105B80005C5C5C5C5C5C5C5C5D5D5D5D5D5D5D5D4D
:105B90005E5E5E5E5E5E5E62666A6E72767A7E8271
:105BA000868A8E92969A9EA2A6AAAEB2B6BABEC2B5
:105BB000C6CACED2D6DADEE2E6EAEEF2F6FAFE02A5
:105BC00060606060606060606161616161616161CD
:105BD0006262626262626262666A6E72767A7E8215
:105BE000868A8E92969A9EA2A6AAAEB2B6BABEC275
:105BF000C6CACED2D6DADEE2E6EAEEF2F6FAFE0265
:105C0000646464646464646465656565656565654C
:105C10006666666666666666676B6F73777B7F83AC
:105C2000878B8F93979B9FA3A7ABAFB3B7BBBFC324
:105C3000C7CBCFD3D7DBDFE3E7EBEFF3F7FBFF0314
:105C400068686868686868686969696969696969CC
:105C50006A6A6A6A6A6A6A6A6B6B6F73777B7F8348
:105C6000878B8F93979B9FA3A7ABAFB3B7BBBFC3E4
:105C7000C7CBCFD3D7DBDFE3E7EBEFF3F7FBFF03D4
:105C80006C6C6C6C6C6C6C6C6D6D6D6D6D6D6D6D4C
:105C90006E6E6E6E6E6E6E6E6F6F6F73777B7F83E0
:105CA000878B8F93979B9FA3A7ABAFB3B7BBBFC3A4
:105CB000C7CBCFD3D7DBDFE3E7EBEFF3F7FBFF0394
:105CC00070707070707070707171717171717171CC
:105CD000727272727272727273737373777B7F8374
:105CE000878B8F93979B9FA3A7ABAFB3B7BBBFC364
:105CF000C7CBCFD3D7DBDFE3E7EBEFF3F7FBFF0354
:105D0000747474747474747475757575757575754B
:105D1000767676767676767677777777777B7F8303
:105D2000878B8F93979B9FA3A7ABAFB3B7BBBFC323
:105D3000C7CBCFD3D7DBDFE3E7EBEFF3F7FBFF0313
:105D400078787878787878787979797979797979CB
:105D50007A7A7A7A7A7A7A7A7B7B7B7B7B7B7F838F
:105D6000878B8F93979B9FA3A7ABAFB3B7BBBFC3E3
:105D7000C7CBCFD3D7DBDFE3E7EBEFF3F7FBFF03D3
:105D80007C7C7C7C7C7C7C7C7D7D7D7D7D7D7D7D4B
:105D90007E7E7E7E7E7E7E7E7F7F7F7F7F7F7F8317
:105DA000878B8F93979B9FA3A7ABAFB3B7BBBFC3A3
:105DB000C7CBCFD3D7DBDFE3E7EBEFF3F7FBFF0393
:105DC00080808080808080808181818181818181CB
:105DD000828282828282828283838383838383839B
:105DE000878B8F93979B9FA3A7ABAFB3B7BBBFC363
:105DF000C7CBCFD3D7DBDFE3E7EBEFF3F7FBFF0353
:105E0000848484848484848485858585858585854A
:105E1000868686868686868687878787878787871A
:105E200003070B0F13171B1F23272B2F33373B3F62
:105E300043474B4F53575B5F63676B6F73777B7F52
:105E400088888888888888888989898989898989CA
:105E50008A8A8A8A8A8A8A8A8B8B8B8B8B8B8B8B9A
:105E60000703070B0F13171B1F23272B2F33373B5A
:105E70003F43474B4F53575B5F63676B6F73777B52
:105E80008C8C8C8C8C8C8C8C8D8D8D8D8D8D8D8D4A
:105E90008E8E8E8E8E8E8E8E8F8F8F8F8F8F8F8F1A
:105EA0000B0703070B0F13171B1F23272B2F33374A
:105EB0003B3F43474B4F53575B5F63676B6F737752
:105EC00090909090909090909191919191919191CA
:105ED000929292929292929293939393939393939A
:105EE0000F0B0703070B0F13171B1F23272B2F3332
:105EF000373B3F43474B4F53575B5F63676B6F7352
:105F00009494949494949494959595959595959549
:105F10009696969696969696979797979797979719
:105F2000130F0B0703070B0F13171B1F23272B2F11
:105F300033373B3F43474B4F53575B5F63676B6F51
:105F400098989898989898989999999999999999C9
:105F50009A9A9A9A9A9A9A9A9B9B9B9B9B9B9B9B99
:105F600017130F0B0703070B0F13171B1F23272BE9
:105F70002F33373B3F43474B4F53575B5F63676B51
:105F80009C9C9C9C9C9C9C9C9D9D9D9D9D9D9D9D49
:105F90009E9E9E9E9E9E9E9E9F9F9F9F9F9F9F9F19
:105FA0001B17130F0B0703070B0F13171B1F2327B9
:105FB0002B2F33373B3F43474B4F53575B5F636751
:105FC000A0A0A0A0A0A0A0A0A1A1A1A1A1A1A1A1C9
:105FD000A2A2A2A2A2A2A2A2A3A3A3A3A3A3A3A399
:105FE0001F1B17130F0B0703070B0F13171B1F2381
:105FF000272B2F33373B3F43474B4F53575B5F6351
:10600000A4A4A4A4A4A4A4A4A5A5A5A5A5A5A5A548
:10601000A6A6A6A6A6A6A6A6A7A7A7A7A7A7A7A718
:10602000231F1B17130F0B0702060A0E12161A1E48
:1060300022262A2E32363A3E42464A4E52565A5E60
:10604000A8A8A8A8A8A8A8A8A9A9A9A9A9A9A9A9C8
:10605000AAAAAAAAAAAAAAAAABABABABABABABAB98
:1060600027231F1B17130F0B0602060A0E12161A00
:106070001E22262A2E32363A3E42464A4E52565A60
:10608000ACACACACACACACACADADADADADADADAD48
:10609000AEAEAEAEAEAEAEAEAFAFAFAFAFAFAFAF18
:1060A0002B27231F1B17130F0A0602060A0E1216B0
:1060B0001A1E22262A2E32363A3E42464A4E525660
:1060C000B0B0B0B0B0B0B0B0B1B1B1B1B1B1B1B1C8
:1060D000B2B2B2B2B2B2B2B2B3B3B3B3B3B3B3B398
:1060E0002F2B27231F1B17130E0A0602060A0E1258
:1060F000161A1E22262A2E32363A3E42464A4E5260
:10610000B4B4B4B4B4B4B4B4B5B5B5B5B5B5B5B547
:10611000B6B6B6B6B6B6B6B6B7B7B7B7B7B7B7B717
:10612000332F2B27231F1B17120E0A0602060A0EF7
:1061300012161A1E22262A2E32363A3E42464A4E5F
:10614000B8B8B8B8B8B8B8B8B9B9B9B9B9B9B9B9C7
:10615000BABABABABABABABABBBBBBBBBBBBBBBB97
:1061600037332F2B27231F1B16120E0A0602060A8F
:106170000E12161A1E22262A2E32363A3E42464A5F
:10618000BCBCBCBCBCBCBCBCBDBDBDBDBDBDBDBD47
:10619000BEBEBEBEBEBEBEBEBFBFBFBFBFBFBFBF17
:1061A0003B37332F2B27231F1A16120E0A0602061F
:1061B0000A0E12161A1E22262A2E32363A3E42465F
:1061C000C0C0C0C0C0C0C0C0C1C1C1C1C1C1C1C1C7
:1061D000C2C2C2C2C2C2C2C2C3C3C3C3C3C3C3C397
:1061E0003F3B37332F2B27231E1A16120E0A0602A7
:1061F000060A0E12161A1E22262A2E32363A3E425F
:10620000C4C4C4C4C4C4C4C4C5C5C5C5C5C5C5C546
:10621000C6C6C6C6C6C6C6C6C7C7C7C7C7C7C7C716
:10622000433F3B37332F2B27221E1A16120E0A0626
:106230000105090D1115191D2125292D3135393D6E
:10624000C8C8C8C8C8C8C8C8C9C9C9C9C9C9C9C9C6
:10625000CACACACACACACACACBCBCBCBCBCBCBCB96
:1062600047433F3B37332F2B26221E1A16120E0AA6
:10627000050105090D1115191D2125292D31353966
:10628000CCCCCCCCCCCCCCCCCDCDCDCDCDCDCDCD46
:10629000CECECECECECECECECFCFCFCFCFCFCFCF16
:1062A0004B47433F3B37332F2A26221E1A16120E26
:1062B00009050105090D1115191D2125292D313556
:1062C000D0D0D0D0D0D0D0D0D1D1D1D1D1D1D1D1C6
:1062D000D2D2D2D2D2D2D2D2D3D3D3D3D3D3D3D396
:1062E0004F4B47433F3B37332E2A26221E1A1612A6
:1062F0000D09050105090D1115191D2125292D313E
:10630000D4D4D4D4D4D4D4D4D5D5D5D5D5D5D5D545
:10631000D6D6D6D6D6D6D6D6D7D7D7D7D7D7D7D715
:10632000534F4B47433F3B37322E2A26221E1A1625
:10633000110D09050105090D1115191D2125292D1D
:10634000D8D8D8D8D8D8D8D8D9D9D9D9D9D9D9D9C5
:10635000DADADADADADADADADBDBDBDBDBDBDBDB95
:1063600057534F4B47433F3B36322E2A26221E1AA5
:1063700015110D09050105090D1115191D212529F5
:10638000DCDCDCDCDCDCDCDCDDDDDDDDDDDDDDDD45
:10639000DEDEDEDEDEDEDEDEDFDFDFDFDFDFDFDF15
:1063A0005B57534F4B47433F3A36322E2A26221E25
:1063B0001915110D09050105090D1115191D2125C5
:1063C000E0E0E0E0E0E0E0E0E1E1E1E1E1E1E1E1C5
:1063D000E2E2E2E2E2E2E2E2E3E3E3E3E3E3E3E395
:1063E0005F5B57534F4B47433E3A36322E2A2622A5
:1063F0001D1915110D09050105090D1115191D218D
:10640000E4E4E4E4E4E4E4E4E5E5E5E5E5E5E5E544
:10641000E6E6E6E6E6E6E6E6E7E7E7E7E7E7E7E714
:10642000635F5B57534F4B47423E3A36322E2A2624
:10643000211D1915110D09050004080C1014181C54
:10644000E8E8E8E8E8E8E8E8E9E9E9E9E9E9E9E9C4
:10645000EAEAEAEAEAEAEAEAEBEBEBEBEBEBEBEB94
:1064600067635F5B57534F4B46423E3A36322E2AA4
:1064700025211D1915110D09040004080C1014180C
:10648000ECECECECECECECECEDEDEDEDEDEDEDED44
:10649000EEEEEEEEEEEEEEEEEFEFEFEFEFEFEFEF14
:1064A0006B67635F5B57534F4A46423E3A36322E24
:1064B0002925211D1915110D08040004080C1014BC
:1064C000F0F0F0F0F0F0F0F0F1F1F1F1F1F1F1F1C4
:1064D000F2F2F2F2F2F2F2F2F3F3F3F3F3F3F3F394
:1064E0006F6B67635F5B57534E4A46423E3A3632A4
:1064F0002D2925211D1915110C08040004080C1064
:10650000F4F4F4F4F4F4F4F4F5F5F5F5F5F5F5F543
:10651000F6F6F6F6F6F6F6F6F7F7F7F7F7F7F7F713
:10652000736F6B67635F5B57524E4A46423E3A3623
:10653000312D2925211D1915100C08040004080C03
:10654000F8F8F8F8F8F8F8F8F9F9F9F9F9F9F9F9C3
:10655000FAFAFAFAFAFAFAFAFBFBFBFBFBFBFBFB93
:1065600077736F6B67635F5B56524E4A46423E3AA3
:1065700035312D2925211D1914100C08040004089B
:10658000FCFCFCFCFCFCFCFCFDFDFDFDFDFDFDFD43
:10659000FEFEFEFEFEFEFEFEFFFFFFFFFFFFFFFF13
:1065A0007B77736F6B67635F5A56524E4A46423E23
:1065B0003935312D2925211D1814100C080400042B
:1065C00000000000000000000101010101010101C3
:1065D0000202020202020202030303030303030393
:1065E0007F7B77736F6B67635E5A56524E4A4642A3
:1065F0003D3935312D2925211C1814100C080400B3
:10660000000000000000000000000000000000008A
:10661000000000000000000000000000000000007A
:10662000000000000000000000000000000000006A
:106630000000000000000000000000000000000159
:10664000000000000000000000000000000000004A
:10665000000000000000000000000000000000003A
:10666000000000000000000000000000000000002A
:106670000000000000000000000000000000000119
:10668000000000000000000000000000000000000A
:1066900000000000000000000000000000000000FA
:1066A00000000000000000000000000000000000EA
:1066B00000000000000000000000000000000001D9
:1066C00000000000000000000000000000000000CA
:1066D00000000000000000000000000000000000BA
:1066E00000000000000000000000000000000000AA
:1066F0000000000000000000000000000000000199
:106700000000000000000000000000000000000089
:106710000000000000000000000000000000000079
:106720000000000000000000000000000000000069
:106730000000000000000000000000000000000158
:106740000000000000000000000000000000000049
:106750000000000000000000000000000000000039
:106760000000000000000000000000000000000029
:106770000000000000000000000000000000000118
:106780000000000000000000000000000000000009
:1067900000000000000000000000000000000000F9
:1067A00000000000000000000000000000000000E9
:1067B00000000000000000000000000000000001D8
:1067C00000000000000000000000000000000000C9
:1067D00000000000000000000000000000000000B9
:1067E00000000000000000000000000000000000A9
:1067F0000000000000000000000000000000000198
:106800000000000000000000000000000000000088
:106810000000000000000000000000000000000078
:106820000000000000000000000000000000000068
:106830000000000000000000000000000000000157
:106840000000000000000000000000000000000048
:106850000000000000000000000000000000000038
:106860000000000000000000000000000000000028
:106870000000000000000000000000000000000117
:106880000000000000000000000000000000000008
:1068900000000000000000000000000000000000F8
:1068A00000000000000000000000000000000000E8
:1068B00000000000000000000000000000000001D7
:1068C00000000000000000000000000000000000C8
:1068D00000000000000000000000000000000000B8
:1068E00000000000000000000000000000000000A8
:1068F0000000000000000000000000000000000197
:106900000000000000000000000000000000000087
:106910000000000000000000000000000000000077
:106920000000000000000000000000000000000067
:106930000000000000000000000000000000000156
:106940000000000000000000000000000000000047
:106950000000000000000000000000000000000037
:106960000000000000000000000000000000000027
:106970000000000000000000000000000000000116
:106980000000000000000000000000000000000007
:1069900000000000000000000000000000000000F7
:1069A00000000000000000000000000000000000E7
:1069B00000000000000000000000000000000001D6
:1069C00000000000000000000000000000000000C7
:1069D00000000000000000000000000000000000B7
:1069E00000000000000000000000000000000000A7
:1069F0000000000000000000000000000000000196
:106A00000000000000000000000000000000000086
:106A10000000000000000000000000000000000076
:106A20000000000000000000000000000000000066
:106A30000000000000000000000000000000000155
:106A40000000000000000000000000000000000046
:106A50000000000000000000000000000000000036
:106A60000000000000000000000000000000000026
:106A70000000000000000000000000000000000115
:106A80000000000000000000000000000000000006
:106A900000000000000000000000000000000000F6
:106AA00000000000000000000000000000000000E6
:106AB00000000000000000000000000000000001D5
:106AC00000000000000000000000000000000000C6
:106AD00000000000000000000000000000000000B6
:106AE00000000000000000000000000000000000A6
:106AF0000000000000000000000000000000000195
:106B00000000000000000000000000000000000085
:106B10000000000000000000000000000000000075
:106B20000000000000000000000000000000000065
:106B30000000000000000000000000000000000154
:106B40000000000000000000000000000000000045
:106B50000000000000000000000000000000000035
:106B60000000000000000000000000000000000025
:106B70000000000000000000000000000000000114
:106B80000000000000000000000000000000000005
:106B900000000000000000000000000000000000F5
:106BA00000000000000000000000000000000000E5
:106BB00000000000000000000000000000000001D4
:106BC00000000000000000000000000000000000C5
:106BD00000000000000000000000000000000000B5
:106BE00000000000000000000000000000000000A5
:106BF0000000000000000000000000000000000194
:106C00000000000000000000000000000000000084
:106C10000000000000000000000000000000000074
:106C20000000000000000000000000000000000064
:106C30000000000000000000000000000000000153
:106C40000000000000000000000000000000000044
:106C50000000000000000000000000000000000034
:106C60000000000000000000000000000000000024
:106C70000000000000000000000000000000000113
:106C80000000000000000000000000000000000004
:106C900000000000000000000000000000000000F4
:106CA00000000000000000000000000000000000E4
:106CB00000000000000000000000000000000001D3
:106CC00000000000000000000000000000000000C4
:106CD00000000000000000000000000000000000B4
:106CE00000000000000000000000000000000000A4
:106CF0000000000000000000000000000000000193
:106D00000000000000000000000000000000000083
:106D10000000000000000000000000000000000073
:106D20000000000000000000000000000000000063
:106D30000000000000000000000000000000000152
:106D40000000000000000000000000000000000043
:106D50000000000000000000000000000000000033
:106D60000000000000000000000000000000000023
:106D70000000000000000000000000000000000112
:106D80000000000000000000000000000000000003
:106D900000000000000000000000000000000000F3
:106DA00000000000000000000000000000000000E3
:106DB00000000000000000000000000000000001D2
:106DC00000000000000000000000000000000000C3
:106DD00000000000000000000000000000000000B3
:106DE00000000000000000000000000000000000A3
:106DF0000000000000000000000000000000000192
:106E00000000000000000000000000000000000082
:106E10000000000000000000000000000000000072
:106E20000000000000000000000000000000000062
:106E30000000000000000000000000000000000052
:00000001FF
